:10010000E4F590C2D5D2D47820C2D47820C2D47578
:100110009850758920758DFD858D8B75B81075A8E3
:1001200092758850120143FAFBF590F4F58CEB20A0
:10013000D5040302013723FBF5901201436A60EEF8
:100140006A80E4E5A022C0E0B2D5EAF4F58CD0E004
:1001500032C0E0C0D0C29875D010E599F5F0640DBA
:100160007010741FC398F46013FBE418F2DBFC02F8
:10017000017C743FC3984004E5F0F208D0D0D0E091
:01018000324C
:020000002100DD
:02002300215169
:02000B0021468C
:00000001FF
